:1000000088C0B0C0AFC0AEC0ADC0B1C0ABC0AAC0A8
:10001000A9C0A8C0A7C0A6C0A5C0A4C0A3C0814550
:1000200086468B479048944997609B619E62A16386
:10003000A464A765AA66AC67AE68B069B280B481F3
:10004000B682B883BA84BB84BD84FF21000000005F
:100050000000000000000000000023456C98C9FF6C
:10006000040714233764A0FFFFFFFFFFFFFFFFFF1C
:10007000FFFFFF00000000000000000023405F7A47
:10008000B4FFFFFFFFFFFF001400081400080E1468
:100090000004080E14000305080E14000305080AE6
:1000A0000E14000305080A0E1014000305080A0EBA
:1000B0001012140008000E00080E0004080E0003C1
:1000C00005080E000305080A0E0004080E101400AF
:1000D000F3F404080E10121400080A0C0E0F10128C
:1000E0001400080EEE1400020304050004140004BA
:1000F0000E1400040810140004080F111400EEED93
:10010000ECEB140E08040004080E00EBECEDEEF32B
:10011000F41411241FBECFE5D2E0DEBFCDBF20E036
:10012000A0E6B0E001C01D92A738B207E1F7E2E611
:10013000F0E085E5808781E083831482128287E086
:1001400086831182ADE6B0E08EEF15968C931597FD
:100150008DEF17968C93118688E58287612C712C20
:10016000C2D0BCC24DCF1BBC19BC18BC0895189599
:1001700025B7277E25BF29B7226029BF21E022BFEE
:10018000019728F020E188952150E9F7F9CF0895EB
:1001900088EE93E0EDCF8CE287B986EC86B9369A8B
:1001A0003699FECF8FEF809360000895369A369986
:1001B000FECF95B18091600089270895CF93C72D18
:1001C00081E0870D8F73782E662D90E079D26FEFE6
:1001D0008C2F90E0CF9174C2FF920F931F93CF9317
:1001E000DF93F82E0CE610E0C5E7D0E081E0F812CE
:1001F00005C0F8016081CE0163D204C0CE0158D29F
:10020000F8018083015011092196CF37D10571F78C
:10021000DF91CF911F910F91FF900895CFDF81E083
:10022000DBCF811101C09FCF815090E0FC01E45BE6
:10023000FF4FE491EBBDFC01E05AFF4FE491E9BDB3
:10024000FC01EC58FF4F849188BD08950F931F93D4
:10025000CF93C82F8B01CC2359F085E0E2DFC80192
:1002600087DF81DFC80184DFC80182DFC150F3CF9F
:10027000CF911F910F910895EF92FF920F931F93CB
:10028000CF93C8E0E82EF12C062F10E084E1C9DFFF
:10029000C7016EDF68DFC8016BDFC150B9F7CF91CE
:1002A0001F910F91FF90EF9008951F93CF93DF93CD
:1002B0008FEA87B986EC86B91092600010E1C0E041
:1002C000D0E085E090E054DF71DFC80FD11D115000
:1002D000C1F7CE0124E0969587952A95E1F7DF9145
:1002E000CF911F91089583EA87B986EC86B9369934
:1002F000FECF369A3699FECFC5B18FE384BBBB9A49
:10030000C39AB99AB89ABC9A81E08ABD83BF9AB55C
:1003100090629ABD9AB590689ABD9FEF9DBD80BFCF
:1003200080E68CBD97B328B3892F90E08095909597
:100330008B7F822B88BB85B7806285BF789487E7E7
:1003400090E0B6D1853511F069DF11C0712C872D91
:1003500090E0AED1682E8F3F19F080E03DDF07C0FE
:10036000872D91E0970D792E803488F3F6CF809118
:100370006B0000916500F0906600109163001123FE
:1003800019F0F12C00E088E18F5F90E040E050E050
:1003900068E870E0882379F09B012F5F3F4FF901F7
:1003A0003197E491EE2319F0922F961BF6CF8150EE
:1003B000AB01B901EFCF892F602F70E0A92FB0E01A
:1003C000E82FF0E0FF2021F09D012E1B3F0B05C020
:1003D0009F0121503109260F371F3197E40FF51F78
:1003E000E4902A583F4FF901E082815049F7900F7D
:1003F00090936100002371F0FF2029F0292F30E055
:100400002150310902C020E030E0F901EA58FF4FE5
:1004100081E0808387E0890F282F2150E22FE91B9C
:10042000F0E0E55FFE4FE491A22FB0E0AA58BF4F85
:10043000EC932913F2CFE82FF0E0EB58FF4F21E0C7
:10044000409176003081431320E0821B282F809357
:100450008600862D853F70F5C93F60F08F5F682E5E
:10046000891708F0612C809187008F5F8F718093CE
:10047000870020C010928700C33DB0F03091680023
:10048000332311F0112331F08F5F682E891790F01C
:10049000612C10C06916E1F3662019F08150682EB6
:1004A00009C02150622E06C01111F2CF8091640064
:1004B000882371F383DE6FDEC62DC53F28F4D0E0BC
:1004C000CA58DF4FC881DC2F10E000E0EE24E3942F
:1004D00080918700803190F15BDE10928700C3E647
:1004E000D0E0C12CD12C81E08C0DFFEFCF1ADF0AB8
:1004F00098819F3F31F4219688E0C816D10499F77E
:1005000018C06DE570E0A2DEF601E359FF4F608090
:1005100088818E25888382DE6FE070E080E296DE3F
:1005200088818E2588837ADE33DE8091630088237C
:1005300011F3612CC0917600DC2F8EC0CE3E19F4F1
:1005400063E481E204C0CD3E21F468E284E194DEFC
:1005500083C0CC3E11F469E203C0CB3E19F462E5DE
:1005600081E0F5CFC33F41F484E15BDE8AE090E0B7
:10057000FFDD88E056DE3DC0C43F59F584E690E0DB
:10058000F7DD09DE13DE90E0292F30E0F901E25EAD
:10059000FF4FE491E81710F49E5FF6CFF901E15E9A
:1005A000FF4FF4906DE770E08F2D829586958770F0
:1005B0004DDE8EEE92E0DCDD65E070E081E046DE4F
:1005C00085E694E0D5DD6DE770E08F2D8F713EDE1E
:1005D0000FC0CE3F81F4612CF12CF0926B001EDE37
:1005E0006AEF70E081E032DEF39498E1F912F5CF22
:1005F000CFDDCEDD31C0CD3F91F4612C8FEF809304
:100600006C000CDE85E00DDEC3DDC2DD84E109DEB9
:100610004CDE80936C0002DEBBDDBADDF9CF8D2F9E
:1006200000DE43DE20916C00821738F00F5F093046
:1006300078F0D33068F0D1500AC090E030E022501A
:100640003109821793071CF4DC1708F4DF5F00E020
:10065000A2DD84EF91E08CDD10928700A7DD803968
:1006600090F41F5F183008F433CFD53120F010E03C
:10067000DAE0CAE02DCFD23040F08D2F86958695F6
:10068000D695D80FCD2F10E023CF6DDD85B7877EAF
:10069000806185BFF89485B7846885BF8B7F85BFEF
:1006A00085B7806285BF889585B78F7D85BFEACF86
:1006B000E199FECF9FBB8EBBE09A99278DB3089539
:1006C000262FE199FECF1CBA9FBB8EBB2DBB0FB668
:1006D000F894E29AE19A0FBE01960895F894FFCF3C
:00000001FF
